:1000000024202C226923052800289408031D152884
:100010007823BF236523F222F522F822FB227823DE
:10002000152319231D23212305286923BF236523B5
:10003000782378232020BF23940803190828162842
:10004000A5228F199E22080083160C308500860198
:1000500083128501051686010D30840024308C0042
:100060008001840A8C0B30281F3084009701170808
:1000700025228000840A970A05301706031D3728B9
:1000800094209030A400A500A600A70008008207D5
:100090003334333432342C3406340C3401340234E7
:1000A0000C0882070034013402340334043405346C
:1000B00006340734083409340A340B340C340D3454
:1000C0000E340F34820708294029C2296C291629C9
:1000D0005029D629832924295A29EA299A293229FB
:1000E0006329FB29AE298207A628CC28EF288F1880
:1000F00008009408031D08008F140430900040305D
:100100008F060F1F362A692394203622C030922290
:100110002730FF288F1808008F1404309000942097
:100120001408940A0F13732860309B009C009D00F4
:100130009E00231C1B16A31C1C16231D1D16A31D8D
:100140001E16AC01AD01AE01AF0108008030922255
:100150000530FF20C030922241307A2264307A226A
:1001600064307A2272307A222030231C60307A2266
:100170001F0888222030A31C60307A2220088822A1
:100180002030231D60307A22210888222030A31DD0
:1001900060307A222208882A803092221630FF208E
:1001A000C030922243307A2256307A223A307A2274
:1001B0002C08AE00AF00013E8C222D307A222D0893
:1001C0008C2263230310AE0C03102E0C013EAE00F4
:1001D00088222D307A222C080339AF00882A9420F7
:1001E000940197011F30840000088C0017080C222E
:1001F000840A970A05301706031DF428362A97004B
:10020000170825228E08031908007A22970A002968
:1002100014180F291030231C9B06A406080024166E
:100220000130A3061B12231C1B16AA2814181D2913
:100230001030A31C9C06A506080025160230A30654
:100240001C12A31C1C16AA2814182B291030231DBD
:100250009D06A606080026160430A3061D12231DBF
:100260001D16AA28141839291030A31D9E06A706AA
:10027000080027160830A3061E12A31D1E16AA2862
:100280009418452920309B06080069232E08910008
:100290002523692336236923013091002523692B07
:1002A0009418552920309C06080069232C08AF00BB
:1002B0003623692B94185F2920309D060800692396
:1002C0005E235E23692B9418682920309E0608005F
:1002D000692349234923692B14187E2994188129FD
:1002E0001F30231C0F302C0603190800AC0A231CF6
:1002F0007C2910309B061B1E9B0A08009F0AAA201F
:100300000800AC0AD02814189529941898291F3091
:10031000A31C0F302D0603190800AD0AA31C932956
:1003200010309C061C1E9C0A0800A00AAA20080087
:10033000AD0AD0281418AC29941808001F30231DCA
:100340000F302E0603190800AE0A231DAA2910300B
:100350009D061D1E9D0A0800A10AAA281418C0297E
:10036000941808001F30A31D0F302F060319080032
:10037000AF0AA31DBE2910309E061E1E9E0A08004D
:10038000A20AAA281418D1299418D4292C080319D0
:100390000800AC03231CCF2910309B061B1A9B03BB
:1003A00008009F03AA200800AC03D0281418E529F0
:1003B0009418E8292D0803190800AD03A31CE329AC
:1003C00010309C061C1A9C030800A003AA200800F9
:1003D000AD03D0281418F929941808002E08031921
:1003E0000800AE03231DF72910309D061D1A9D033A
:1003F0000800A103AA2814180A2A941808002F0834
:1004000003190800AF031030A31D082A9E061E1A08
:100410009E030800A203AA288D0025220C060319BA
:1004200008000D0889008316081583120C0888003F
:10043000831655308900AA3089008814081E1E2AA8
:100440000811081283120B13080089008316081480
:10045000831208088E00080096229701950117085C
:1004600047207A22970A971D2F2A962280309222BF
:100470004C307A226F307A2263307A223A307A22F4
:100480001F0888222D30241A2A307A222008882238
:100490002D30251A2A307A22210888222D30261A5A
:1004A0002A307A22220888222D30271A2A307A22EE
:1004B000C03092227E309B1E7F307A222C088C2204
:1004C0007E309C1E7F307A222D088C227E309D1E2D
:1004D0007F307A222E088C227E309E1E7F307A2238
:1004E0002F088C2A9300130E0F3930387A22130804
:1004F0000F393038920014308C008C0B7D2A80220A
:10050000920E12080F391504860085148510080014
:100510009A00D1230E08722A9A00D1230D0878225E
:100520000E08722A15127A221516080014308C0053
:1005300096309700ED238C0B982A08001108622052
:100540008F119408031936220800051D7728851D90
:100550008A288F1CAF2A900B08008F1008000F1BF1
:100560000800E122EF308D0006080B108D0C031CF3
:10057000CA2A0D08860000000B1CB42A0F18C92ACD
:100580000F14060E8E00CC2291008F158F140430AC
:100590009000EB2A0F10C92A8C018D1DD62A8C0AD7
:1005A0000D1DD62A8C0A8D1CD62A8C0A0E1C5028AA
:1005B0008E1CDF2A0E1DDD2A0C158C1550280C15FB
:1005C000502806089600FF30860083168113F0300D
:1005D000860083120800160886008316811786019C
:1005E000831208008923FE22092B892300230B2B69
:1005F000892302230D2B892304230F2B1F08052B8E
:100600002008052B2108052B2208A8009900982313
:10061000BF2B1B08102B1C08102B1D08102B1E08AD
:10062000A90099009823BF23A62B8923FE22240822
:10063000102B892300232508102B89230223260849
:10064000102B892304232708102B063092008923BE
:100650007D309900A8009823BF231108A9009900B4
:100660009823BF23A623920B272B08000630920065
:1006700089232F087F3978389900A8009823BF2351
:100680002D08A90099009823BF23A623920B382B8D
:10069000080089239901A8019823BF23EC30A90001
:1006A00099009823BF232C08AA0099009823BF2300
:1006B0002D08AB0099009823BF23A62B8723A901FF
:1006C0007C30A800502B20307A2A05120000051635
:1006D00008001430920089239901A801A9019823E8
:1006E000BF2399019823BF23A623920B6B2B0800ED
:1006F0008923FF309900A80098237E2B7F2B802B25
:100700000000BF239901A9019823BF23A62B19300C
:100710008A2B0F308C000000000000000000000059
:10072000B3238C0B8B2B942B952B962B0000BF2B7C
:1007300008309A000310991FA42BB3230000000077
:10074000990D9A0B9B2B0800BF23A02B2808290684
:100750002A062B0699009823B323AA01AB0194081B
:1007600003192020BF2B0000000003309700ED2369
:10077000CE230000000004309700ED23CE2B0000B4
:100780000000000007309700ED23CE230830000062
:100790000000000000009700ED23CE2B01308506FD
:1007A00008000310083099008D018E019A0D8E0DFE
:1007B0008D0D990BDC2B00340E30E1230D30E1233D
:1007C000D62B8400033000078C008C198000303059
:1007D00000078C008C1B800000340000000000002B
:1007E0000000000001309800000000000000980B9D
:0807F000F42B970BF22B0034EF
:02400E00F93F78
:1042000003000400050006000F0053007400610065
:1042100074006E00230031002000230032002000D3
:104220002300330020002300340000005300650009
:104230007200760020004D006F00640065002000D1
:104240005000610067002F0052006700000020004E
:1042500045006D0065007200670065006E00630038
:1042600079002000530074006F00700021000000EE
:00000001FF
